:020000020000FC
:02000000D2C06C
:0200040018954D
:02000800189549
:02000C0091C0A1
:02001000189541
:0200140018953D
:02001800189539
:02001C0041C0E1
:02002000189531
:0200240018952D
:02002800189529
:02002C00189525
:02003000189521
:0200340018951D
:0200380017C0EF
:02003C00189515
:02004000189511
:0200440018950D
:020048008AC06C
:02004C0096C05C
:020054001895FD
:020058001895F9
:02005C001895F5
:020060001895F1
:020064001895ED
:100068002FB611964423A1F04A3021F42B984A95D3
:100078002FBE1895413041F070FE2B9870FC2B9ADA
:1000880076944A952FBE18952B9A4A952FBE1895A7
:100098002B9A0E7F2FBE18952FB61A9519F418E0D3
:1000A80055273A95393091F4123041F0113011F456
:1000B8002FBE1895189953952FBE189518995395D2
:1000C800543008F0086022272FBE1895332391F08A
:1000D800123041F0113011F42FBE1895189953952C
:1000E8002FBE1895269518995395543008F0206816
:1000F8002FBE189503FD0DC0123010F02FBE1895B5
:10010800DC2DCD2D2993D53011F4D1E0C0E2CD2ED0
:10011800DC2E2227332718E077277093B1007093DD
:100128007000057F2FBE18951899189501FD189530
:1001380003FD18952FB6026077E07093B30072E064
:100148007093B10072E07093700039E02227552750
:1001580018E02FBE18952FB67091C600D82DC92D5E
:100168007993D93010F0D5E0C0E08D2E9C2E2FBEAB
:1001780018952FB6C02DC13051F0C23021F0309201
:10018800C6000A940AC04092C6000A9406C070913C
:10019800C1007F7D7093C10000242FBE1895F8948C
:1001A80091E09EBF9CE19DBFAA27BB27992794B9E0
:1001B80097B99AB99FEF95B998B99BB9259A249A96
:1001C800529A2D9A2C9A539A5B985A98239A2B9A5A
:1001D80009B10095007C90B7906890BF97E097BDF3
:1001E80092E094BD93E095BD92E090936E0097E005
:1001F8009093B30092E09093B00092E09093B10096
:1002080092E09093700095E0892EA92E90E0992EA7
:10021800B92E99279093C500802F807C882311F4EC
:1002280099E109C0803411F493E305C0803811F4D2
:1002380097E601C09FEC9093C40098E99093C100A1
:1002480091E0C92EE92E90E2D92EF92E91E09093F3
:100258006B0091E090936800772444272227332786
:100268000024112466278EE19EE08093600090931D
:10027800600078948827DAD08A95E9F739D000FDAC
:100288002BC065D04EF54D9924C0892F8A3021F1B5
:100298008D3011F0803241F4662321F0712C4AE050
:1002A80001606627112418C0813608F08052982F03
:1002B80084D056F46395633038F4812D8295807F1D
:1002C8009F70982B192E08C08FE386D011246627BB
:1002D80003C0792E4AE00160002081F653D076F6FB
:1002E800892F4D9902C088D0C9CF76D0C7CFC6CF45
:1002F800A8958B2D9A2D891949F0980908F49C5FC7
:10030800992321F4803220F0803418F05A9801C0E3
:100318005A9AB430D9F4F894000000000000BB27C2
:10032800AA27789499B19095907C802F807C891722
:1003380019F02D982C98FDCF552019F05A9409F4EE
:100348002D9A662019F06A9409F42C9A0895F89465
:100358009B1429F48A1419F47894E8940895FA2DD2
:10036800EB2D9191F93010F0F5E0E0E0AF2EBE2EC4
:100378007894983F29F09E3F19F02D98E8E05E2E7A
:1003880068940895F894DF1429F4CE1419F4789435
:10039800E8940895FE2DEF2D9191F53011F4F1E0D8
:1003A800E0E2EF2EFE2E7894983F29F09E3F19F058
:1003B8002C98E8E06E2E68940895913420F09734D4
:1003C80048F4975305C0903328F090539A3010F4AE
:1003D80068940895E89408959F939091C00095FFBC
:1003E800FCCF8093C600002403949091C1009062D2
:1003F8009093C1009F9108958F9380E2EDDF8F91D4
:100408008F9382958F70805D8A3308F0895F80337F
:1004180011F402C080E2E0DF8F918F938F70805DCE
:100428008A3308F0895FD8DF8F9108959F9397E109
:080438009A95F1F79F910895D8
:00000001FF
